:020000040000FA
:100000006C28831600308600831286010800FE30BB
:1000100067203830860086110A3067203830860025
:10002000861102306720383086008611372028304C
:100030008600861137202830860086118830860099
:1000400086113720083086008611F8308600861128
:100050003720083086008611183086008611372038
:1000600008308600861168308600861108008316E5
:10007000F030860083120615861086150608861154
:10008000061586108615000086118039031D372855
:10009000061183160030860083120800C8308600DF
:1000A00086110830860086110800A000372020083D
:1000B000F0390A3886008611200EF0390A38860099
:1000C00086110800A530A100A10B64280800A20039
:1000D0006220A20B68280800012007204830552024
:1000E000453055204C3055204C3055204F30552050
:1000F00020305520573055204F3055205230552054
:100100004C30552044305520213055204E204C3065
:100110005520493055204E3055204530552020304F
:0A01200055203230552000009328CE
:00000001FF
